:1000000002091B750A03E4F509FB7A0079097F01EF
:10001000120046750A03E4F509FB7A0079097F03AB
:100020000200460208AA7DA37C08ED1D70011C1485
:0D0030004C70F7EF1F70011E144E70EA2295
:100043000207BEEFD394077480948040037FFF229E
:10005300120531FED394037480948040037FFF2202
:10006300EF7044EE700B90000112054AF452935264
:10007300941205316401700B90000112054A4293FA
:10008300F45294120531FE6402700A9000011205C5
:100093004A42934294EE6403700D90000112054AA4
:1000A300FEF45293EE4294EF64017046120531FE62
:1000B300700B90000112054AF452915292EE6401C2
:1000C300700B90000112054A4291F45292120531CD
:1000D3006402700A90000112054A4291429212058D
:1000E300316403700D90000112054AFEF45291EE43
:1000F3004292EF64027046120531FE700B900001CC
:1001030012054AF452955296EE6401700B90000169
:1001130012054A4295F452961205316402700A9010
:10012300000112054A429542961205316403700D8F
:1001330090000112054AFEF45295EE4296EF6403D5
:100143007046120531FE700B90000112054AF452FD
:10015300B152B2EE6401700B90000112054A42B134
:10016300F452B21205316402700A90000112054A7A
:1001730042B142B21205316403700D9000011205C1
:100183004AFEF452B1EE42B2EF64047046120531F6
:10019300FE700B90000112054AF452B352B4EE64A0
:1001A30001700B90000112054A42B3F452B41205D8
:1001B300316402700A90000112054A42B342B4123C
:1001C30005316403700D90000112054AFEF452B329
:1001D300EE42B4EF64057046120531FE700B9000D9
:1001E3000112054AF452C952CAEE6401700B900021
:1001F3000112054A42C9F452CA1205316402700A57
:1002030090000112054A42C942CA120531640370C3
:100213000D90000112054AFEF452C9EE42CAEF6482
:10022300067046120531FE700B90000112054AF468
:1002330052CB52CCEE6401700B90000112054A427E
:10024300CBF452CC1205316402700A9000011205FE
:100253004A42CB42CC1205316403700D9000011267
:10026300054AFEF452CBEE42CCEF64077049120507
:1002730031FF7E00700B90000112054AF452E152E7
:10028300E2EF64014E700B90000112054A42E1F463
:1002930052E21205316402700A90000112054A42CB
:1002A300E142E21205316403700D90000112054A28
:1002B300FFF452E1EF42E27F00228F128B138A1484
:1002C3008915EF64016003020430751B01F51CF509
:1002D3001DF51EF51FF520F521F516C3E5169480CF
:1002E30074809480501174002516F582E43401F56E
:1002F30083E4F0051680E4E4F516C3E516948074F0
:10030300809480501174002516F582E43400F5833F
:10031300E4F0051680E4AB13AA14A915120531FF06
:10032300E598543F4FF598EF64C06008EF64406070
:10033300030203DF9000021206697F007E607D5492
:100343007C001205B38F1A8E198D188C17E4FFFEEB
:100353007D01FCAB1AAA19A918A817C312064540B8
:10036300037FFF22C3E4951AF51AE49519F519746E
:10037300019518F518E49517F517AB13AA14A915E9
:1003830090000112054A64027026538EEF438E01DA
:10039300538EF7438E04AF1AAE19AD18AC17780815
:1003A3001206568FD6851AD753AFFB438E1080663D
:1003B300C28E538EFE5389BF5389CF438E40AF1AEB
:1003C300AE19AD18AC1778081206568F8D851A8BA7
:1003D300C2AB5389BF538FFDD28E803AAB13AA149D
:1003E300A915120531FF7E00701490000812054A0A
:1003F30064017005438E20801D538EDF8018EF64E7
:10040300804E701290000812054A640170054387FC
:1004130080800353877FAB13AA14A915900007129A
:10042300054A7004C29C8002D29C7F0022E51264BC
:1004330002600302052E752202F523F524F525F546
:1004430026F527F528F516C3E51694807480948065
:10045300501174802516F582E43401F583E4F00528
:100463001680E4E4F516C3E51694807480948050F6
:100473001174802516F582E43400F583E4F0051643
:1004830080E4AB13AA14A915120531FF7E0064C0E2
:100493006005EF64407077EF64C04E7005439A8047
:1004A3008003539A7F9000021206697F007E607D6D
:1004B300547C001205B38F1A8E198D188C17E4FF24
:1004C300FE7D01FCAB1AAA19A918A817C312064589
:1004D30040037FFF22C3E4951AF51AE49519F51931
:1004E30074019518F518E49517F517538EEF538E8D
:1004F300F7438E04AF1AAE19AD18AC17780812067D
:10050300568FD6851AD753AFFB438E1080037FFFD8
:1005130022AB13AA14A91590000712054AC454F07C
:10052300FFE59A54EF4FF59A7F00227FFF22BB012C
:100533000689828A83E0225002E722BBFE02E3227D
:1005430089828A83E49322BB010CE58229F582E543
:10055300833AF583E0225006E92582F8E622BBFEC2
:1005630006E92582F8E222E58229F582E5833AF558
:1005730083E4932275F008758200EF2FFFEE33FEBC
:10058300CD33CDCC33CCC58233C5829BED9AEC9968
:10059300E58298400CF582EE9BFEED9AFDEC99FC0A
:1005A3000FD5F0D6E4CEFBE4CDFAE4CCF9A8822251
:1005B300B800C1B90059BA002DEC8BF084CFCECD71
:1005C300FCE5F0CBF97818EF2FFFEE33FEED33FDAA
:1005D300EC33FCEB33FB10D703994004EB99FB0F8F
:1005E300D8E5E4F9FA227818EF2FFFEE33FEED3366
:1005F300FDEC33FCC933C910D7059BE99A4007ECDE
:100603009BFCE99AF90FD8E0E4C9FAE4CCFB227524
:10061300F010EF2FFFEE33FEED33FDCC33CCC833B8
:10062300C810D7079BEC9AE899400AED9BFDEC9A1A
:10063300FCE899F80FD5F0DAE4CDFBE4CCFAE4C892
:10064300F922EB9FF5F0EA9E42F0E99D42F0E89C27
:1006530045F022E8600FECC313FCED13FDEE13FE2F
:10066300EF13FFD8F122BB010DE58229F582E58363
:100673003AF5830206A65007E92582F8020699BBDC
:10068300FE07E92582F80206B2E58229F582E583B1
:100693003AF5830206BFE6FB08E6F908E6FA08E640
:1006A300CBF822E0F8A3E0F9A3E0FAA3E0FB22E20F
:1006B300FB08E2F908E2FA08E2CBF822E493F874C3
:1006C3000193F9740293FA740393FB221200031249
:1006D300076DD2AF7BFF7A09793B1208F57BFF7A6E
:1006E3000979581209087F017E00120026D3E520FC
:1006F30094007480948040321520E520702CD3E55B
:100703001F940074809480401EE4F508E508C395A7
:100713001F501474002508F582E43400F583E0FFCC
:10072300120927050880E5E4F51FD3E52794007433
:1007330080948040B11527E52770ABD3E52694005C
:1007430074809480401EE4F508E508C39526501490
:1007530074802508F582E43400F583E0FF12093143
:10076300050880E5E4F5260206E9750940750A01E6
:10077300750E00750DC2750C01750B00751001E443
:10078300F511FB7A0079097F011202BD7D017F011A
:1007930012085D750940E4F50E750DE1F50CF50BD6
:1007A300751001FB7A0079097F021202BD7D017F7A
:1007B3000112080F53A23F53BAFE22C0E0C083C008
:1007C30082C0D075D000C007E59A30E029539AFE65
:1007D300E5287022C3E526948074809480400375D5
:1007E3002600AF26052674802FF582E43400F583B6
:1007F300E59BF0752705E59A30E106539AFD7525CB
:1008030000D007D0D0D082D083D0E032EFD3940190
:10081300748094805007E5AF54FE4FF5AFEDFF7E33
:1008230000D3940374809480502DEF700653B6FE6A
:1008330053B5FEEF64014E700653B6FE43B501EFA8
:1008430064024E700643B60153B5FEEF64034E7067
:100853000643B60143B5017F0022EFFBD394017435
:100863008094805009EB7004C2AC8002D2ACEDFFDF
:100873007E00D39403748094805029EF700553B79E
:10088300EFC2BCEF64014E700553B7EFD2BCEF6407
:10089300024E700543B710C2BCEF64034E700543AC
:1008A300B710D2BC7F0022C0E0C083C082C0D07525
:1008B300D000C007309828C298E5217022C3E51FF5
:1008C3009480748094804003751F00AF1F051F74CC
:1008D300002FF582E43400F583E599F075200530A7
:1008E3009905C299751E00D007D0D0D082D083D08D
:1008F300E032120531FF600C120927740129F9E473
:100903003AFA80EE22120531FF600C1209317401AC
:1009130029F9E43AFA80EE22787FE4F6D8FD75816E
:10092300280206CF8F99751E01E51E70FC228F9B4E
:10093300752501E52570FC22535443382055415257
:10094300543120546573742050726F6772616D6DFA
:1009530065210D0A00535443382055415254322027
:10096300546573742050726F6772616D6D65210DEC
:020973000A0078
:00000001FF
